:020000040000FA
:100000000C945D000C9485000C9485000C94850084
:100010000C9485000C9485000C9485000C9485004C
:100020000C9485000C9485000C9485000C9485003C
:100030000C9485000C9485000C9485000C9485002C
:100040000C942D060C9485000C94FB050C94D5059E
:100050000C9485000C9485000C9485000C9485000C
:100060000C9477060C948500000000080002010043
:100070000003040700000000000000000000000072
:10008000250028002B0000000000240027002A0083
:10009000040404040404040402020202020203032E
:1000A0000303030301020408102040800102040836
:1000B0001020010204081020960711241FBECFEF64
:1000C000D8E0DEBFCDBF11E0A0E0B1E0E0EAFAE1A8
:1000D00002C005900D92A633B107D9F722E0A6E33E
:1000E000B1E001C01D92A53CB207E1F710E0CDE5FB
:1000F000D0E004C02197FE010E94480DCC35D10705
:10010000C9F70E94F6070C944E0D0C94000090E085
:10011000FC01EC55FF4F249180579F4FFC018491C7
:10012000882399F090E0880F991FFC01EA57FF4F50
:10013000A591B491FC01E458FF4F859194918FB73C
:10014000F894EC91E22BEC938FBF089508950895F5
:10015000AF92BF92CF92DF92EF92FF920F931F93D5
:10016000CF93DF936C017B018B01040F151FEB0113
:100170005E01AE18BF08C017D10759F06991D601CA
:10018000ED91FC910190F081E02DC6010995892B3C
:1001900079F7C501DF91CF911F910F91FF90EF90FB
:1001A000DF90CF90BF90AF900895FC01538D448DA8
:1001B000252F30E0842F90E0821B930B541710F012
:1001C000CF96089501970895FC01918D828D98171F
:1001D00061F0A28DAE0FBF2FB11D5D968C91928DF7
:1001E0009F5F9F73928F90E008958FEF9FEF089528
:1001F000FC01918D828D981731F0828DE80FF11DF1
:10020000858D90E008958FEF9FEF0895FC01918D0B
:10021000228D892F90E0805C9F4F821B91098F7304
:100220009927089589EF91E00E94060121E0892B2A
:1002300009F420E0822F089580E090E0892B29F0D6
:100240000E94120181110C9400000895FC01A48DFC
:10025000A80FB92FB11DA35ABF4F2C91848D90E0E8
:1002600001968F739927848FA689B7892C93A089CB
:10027000B1898C91837080648C93938D848D981355
:1002800006C00288F389E02D80818F7D80830895E8
:10029000EF92FF920F931F93CF93DF93EC0181E0D6
:1002A000888F9B8D8C8D98131AC0E889F98980817D
:1002B00085FF15C09FB7F894EE89FF896083E889B0
:1002C000F98980818370806480839FBF81E090E0A2
:1002D000DF91CF911F910F91FF90EF900895F62E2F
:1002E0000B8D10E00F5F1F4F0F731127E02E8C8DC9
:1002F0008E110CC00FB607FCFACFE889F98980810E
:1003000085FFF5CFCE010E942601F1CFEB8DEC0FDA
:10031000FD2FF11DE35AFF4FF0829FB7F8940B8F2A
:10032000EA89FB8980818062CFCFCF93DF93EC0194
:10033000888D8823B9F0AA89BB89E889F9898C91CD
:1003400085FD03C0808186FD0DC00FB607FCF7CF89
:100350008C9185FFF2CF808185FFEDCFCE010E9489
:100360002601E9CFDF91CF91089590E0FC01E85993
:10037000FF4F2491FC01EC55FF4F3491FC01E057F5
:10038000FF4FE491EE23C9F0222339F0233001F12D
:10039000A8F4213019F1223029F1F0E0EE0FFF1F0F
:1003A000E458FF4FA591B4918FB7F894EC91611187
:1003B00026C030953E233C938FBF08952730A9F087
:1003C0002830C9F0243049F7809180008F7D03C028
:1003D000809180008F7780938000DFCF84B58F7706
:1003E00084BDDBCF84B58F7DFBCF8091B0008F774C
:1003F0008093B000D2CF8091B0008F7DF9CF3E2B9B
:10040000DACF8E50806480937C0080917A00806483
:1004100080937A0080917A0086FDFCCF80917800ED
:100420009091790008953FB7F89480919D01909143
:100430009E01A0919F01B091A00126B5A89B05C087
:100440002F3F19F00196A11DB11D3FBFBA2FA92F53
:10045000982F8827BC01CD01620F711D811D911D50
:1004600042E0660F771F881F991F4A95D1F70895BC
:100470008F929F92AF92BF92CF92DF92EF92FF92B4
:100480004B015C010E9413026B017C010E9413026C
:100490006C197D098E099F09683E7340810591059D
:1004A000A8F321E0821A9108A108B10888EEC80ECD
:1004B00083E0D81EE11CF11C81149104A104B10455
:1004C00029F7FF90EF90DF90CF90BF90AF909F9073
:1004D0008F90089520917901260F3327331F213201
:1004E0003105ECF42091CD01FC0190E080E0243056
:1004F00069F082E00895A09179012191AC01475AF9
:100500005E4FA40FB52FB11D2C930196861798F35B
:1005100080917901680F6093790180E0089581E00E
:1005200008951092CD0181E08093CC011092C70113
:1005300061E082E10E94B50161E083E10E94B501C2
:10054000E9EBF0E080818E7F808380818D7F8083E6
:1005500088E48093B80085E48093BC000895CF932D
:10056000DF9391E0909358018823B9F0C091B800CF
:10057000D091BA008091BC008A7B8093BC0060E07F
:1005800082E10E94B50160E083E10E94B5010E9412
:100590009102D093BA00C093B800DF91CF91089533
:1005A0000895E091D4018091D301E81730F4F0E090
:1005B000EB52FE4F808190E008958FEF9FEF0895FA
:1005C0009091D4018091D3012FEF3FEF981748F419
:1005D000E92FF0E0EB52FE4F208130E09F5F9093D7
:1005E000D401C90108958091D3019091D401891B50
:1005F000990B0895CF92DF92EF92FF920F931F9382
:10060000CF93DF937C01CB018A01209157012223F4
:1006100089F0EB016B01C40ED51ECC15DD0569F028
:100620006991D701ED91FC910190F081E02DC70116
:100630000995F3CF642F0E946A02C801DF91CF9120
:100640001F910F91FF90EF90DF90CF900895CF937F
:10065000DF931F92CDB7DEB7698320915701222324
:10066000F9F02091A501203258F021E030E0FC01A2
:100670003383228390E080E00F90DF91CF91089543
:100680008091A601E82FF0E0E95CFE4F998190830C
:100690008F5F8093A6018093A50181E090E0ECCF6D
:1006A00061E0CE0101960E946A02F7CF90E080E0FF
:1006B00008958F929F92AF92BF92CF92DF92EF9266
:1006C000FF920F931F93CF93DF93EC01162F672FA9
:1006D000888199812A8131E0309357012093360136
:1006E0001092A6011092A501DC01ED91FC91019000
:1006F000F081E02D099588819981DC01ED91FC91D3
:100700000190F081E02D612F09950091A50181E014
:10071000013208F09CC0109136010E9413026B0157
:100720007C018091CD0181116CC082E08093CD016C
:1007300081E08093CC018FEF8093CB011092CA01AE
:100740000093C901A7E3B1E0E7EAF1E080E0081314
:1007500096C01092C8018091C801110F182B1093F8
:10076000C8018091C701813009F08DC01092C70186
:100770000E9413026B017C018091C8018093BB0031
:100780008091CF019091D001A091D101B091D2017F
:10079000892B8A2B8B2BA1F00E9413020091CF0191
:1007A0001091D0012091D1013091D2016C197D09B5
:1007B0008E099F09061717072807390708F442C052
:1007C0008091BC0083FDD8CF85EC8093BC000E9453
:1007D00013026B017C018091CD01823009F455C078
:1007E0008091CB018F3F09F472C08091CB018032A0
:1007F00009F46FC08091CB01803309F46CC084E0B0
:1008000026C08091CF019091D001A091D101B091EB
:10081000D201892B8A2B8B2B09F483CF0E941302E0
:100820008090CF019090D001A090D101B090D201E2
:100830006C197D098E099F0986169706A806B906C8
:1008400008F06FCF8091CE010E94AF0285E0109238
:10085000A6011092A501109257018823F1F181E8B9
:100860008AA380E0DF91CF911F910F91FF90EF90CD
:10087000DF90CF90BF90AF909F908F9008959D9103
:1008800091938F5F64CF85EEA0CF8091CF0190913F
:10089000D001A091D101B091D201892B8A2B8B2B51
:1008A00009F499CF0E9413020091CF011091D00159
:1008B0002091D1013091D2016C197D098E099F09D7
:1008C000061717072807390708F085CFBBCF80E048
:1008D000BECF82E0BCCF83E0BACF1AA281E0C2CF04
:1008E000FC0101900020E9F73197AF01481B590B3B
:1008F000BC0189EF91E00C94A8008F929F92AF9277
:10090000BF920F931F93CF93DF93CDB7DEB7A1971D
:100910000FB6F894DEBF0FBECDBF19A2423008F467
:100920004AE08E010F5D1F4F842E912CB12CA12C1B
:10093000A50194010E94260DE62FB901CA01EA30F3
:10094000F4F4E05DD801EE938D01232B242B252BAD
:1009500079F790E080E0109719F0CD010E947004C3
:10096000A1960FB6F894DEBF0FBECDBFDF91CF9139
:100970001F910F91BF90AF909F908F900895E95C69
:10098000E1CF4F925F926F927F928F929F92AF9240
:10099000BF92CF92DF92EF92FF920F931F93CF936C
:1009A0006B017C01742EAC019B010E94210D8823F8
:1009B00099F084E291E0CF911F910F91FF90EF9019
:1009C000DF90CF90BF90AF909F908F907F906F906F
:1009D0005F904F900C94700446015701E894B7F86B
:1009E0002FEF3FEF4FE75FE7C501B4010E94210DF4
:1009F00081110DC02FEF3FEF4FE75FE7C501B40155
:100A00000E94570B18161CF488E291E0D4CF2FEF08
:100A10003FEF4FE75FE4C701B6010E94AF0C181625
:100A20001CF48CE291E0C7CF2FEF3FEF4FE75FEC74
:100A3000C701B6010E94570B87FDF3CF20E030E0DD
:100A4000A901C701B6010E94570B10E000E087FF23
:100A50000AC06DE289EF91E00E9448018C01F7FA2B
:100A6000F094F7F8F094C0E060E070E080E09FE37D
:100A70007C1641F020E030E040E251E40E945C0B43
:100A8000CF5FF6CFA70196010E94EB0A2B013C0134
:100A90000E94CE0B4B015C014AE00E947D047C0168
:100AA000E00EF11ECC23C1F1C501B4010E94FD0B83
:100AB0009B01AC01C301B2010E94EA0A4B015C0137
:100AC0006EE289EF91E00E944801E80EF91EC150E4
:100AD00018F120E030E040E251E4C501B4010E9489
:100AE000B40C2B013C010E94CE0B4B01B12CA12C6C
:100AF0004AE0C501B4010E947D04E80EF91EC5015B
:100B0000B4010E94FD0B9B01AC01C301B2010E9424
:100B1000EA0A4B015C01DBCFC701CF911F910F9116
:100B2000FF90EF90DF90CF90BF90AF909F908F900D
:100B30007F906F905F904F90089585ED8093BC00FB
:100B40008091CF019091D001A091D101B091D201BB
:100B50000796A11DB11D23E0B695A795979587959A
:100B60002A95D1F72091BC0024FD03C01092CD013D
:100B700008954091CF015091D0016091D1017091C1
:100B8000D201452B462B472B69F30097A105B105F0
:100B900041F025E32A95F1F700000197A109B10979
:100BA000E1CF8091CE010C94AF021F920F920FB64D
:100BB0000F9211242F933F934F935F936F937F93E3
:100BC0008F939F93AF93BF93EF93FF9389EF91E040
:100BD0000E942601FF91EF91BF91AF919F918F915C
:100BE0007F916F915F914F913F912F910F900FBE29
:100BF0000F901F9018951F920F920FB60F9211240D
:100C00002F938F939F93EF93FF93E0910902F091BD
:100C10000A028081E0910F02F091100282FD1BC058
:100C20009081809112028F5F8F732091130282173F
:100C300041F0E0911202F0E0E750FE4F958F809373
:100C40001202FF91EF919F918F912F910F900FBE04
:100C50000F901F9018958081F4CF1F920F920FB6BE
:100C60000F9211242F933F938F939F93AF93BF9332
:100C70008091F5019091F601A091F701B091F801F2
:100C800030919C0123E0230F2D3758F50196A11DCB
:100C9000B11D20939C018093F5019093F601A093E0
:100CA000F701B093F80180919D0190919E01A09170
:100CB0009F01B091A0010196A11DB11D80939D01DE
:100CC00090939E01A0939F01B093A001BF91AF911B
:100CD0009F918F913F912F910F900FBE0F901F907A
:100CE000189526E8230F0296A11DB11DD2CF1F92A1
:100CF0000F920FB60F9211242F933F934F935F9350
:100D00006F937F938F939F93AF93BF93EF93FF93D3
:100D10008091B900887F803609F44AC0F0F58832A6
:100D200009F4A7C018F5803109F49BC0B8F48823F2
:100D300009F4F9C0883009F494C0FF91EF91BF9194
:100D4000AF919F918F917F916F915F914F913F9163
:100D50002F910F900FBE0F901F901895883109F4B6
:100D600088C0803251F78093CB0114C0803409F4DD
:100D70009DC040F48033B9F38833F9F68093CB01FA
:100D800085ECB0C0803509F485C0883509F496C07B
:100D9000883499F60E949D05D0CF883909F48CC01B
:100DA00038F5883729F050F4883611F0803729F665
:100DB00083E08093CD0110929B0157C0883809F4DD
:100DC0007BC0803919F0803809F0B7CF80919B0142
:100DD000803208F071C0E0919B0181E08E0F80931A
:100DE0009B018091BB00F0E0E558FE4F80833DC041
:100DF000803B39F0E0F4803A09F479C0883A09F090
:100E00009CCF84E08093CD0110927A0110927901F9
:100E1000E091A101F091A2010995809179018111E0
:100E20000FC081E0809379011092590109C0803C84
:100E300009F4A6CF883C09F4A3CF883B09F07DCF05
:100E4000E0917A0181E08E0F80937A01F0E0E75A19
:100E5000FE4F80818093BB0090917A01809179014F
:100E600029C08091C8018093BB0085EC8093BC00B1
:100E700064CF9091CA018091C901981758F5E0910B
:100E8000CA0181E08E0F8093CA01F0E0E955FE4F60
:100E90008081E9CFE091CA0181E08E0F8093CA0181
:100EA0008091BB00F0E0E955FE4F80839091CA012C
:100EB0008091C9019817C8F285E8D8CFE091CA019E
:100EC00081E08E0F8093CA018091BB00F0E0E9556C
:100ED000FE4F80838091CC0181115CCF81E08093B3
:100EE000C70184EA8093BC001092CD0126CF85EC27
:100EF0008093BC001092CD0180919B01803230F430
:100F0000E0919B01F0E0E558FE4F108260919B015B
:100F100070E0E091A301F091A4018BE791E00995C5
:100F200010929B010ACF1092CB0134CFE9EFF1E090
:100F30001382128248EE53E060E070E044835583F0
:100F40006683778384E091E09183808385EC90E0F1
:100F50009587848784EC90E09787868780EC90E083
:100F6000918B808B81EC90E0938B828B82EC90E074
:100F7000958B848B86EC90E0978B868B118E128EEE
:100F8000138E148EA6E9B2E013961C921E9212974D
:100F900014964D935D936D937C93179786E191E042
:100FA00011969C938E93E2EAF2E0128E138E148EC9
:100FB000158E168E178E10A211A21282B183A083F5
:100FC0001482158216821782118E108E178A168A45
:100FD00013821486158616861786108A118A128A3D
:100FE000138A148A12A285E5858B0895CF93DF9327
:100FF00000D000D000D0CDB7DEB7789484B5826041
:1010000084BD84B5816084BD85B5826085BD85B5AC
:10101000816085BD80916E00816080936E0010922A
:1010200081008091810082608093810080918100A5
:101030008160809381008091800081608093800036
:101040008091B10084608093B1008091B000816094
:101050008093B00080917A00846080937A008091C0
:101060007A00826080937A0080917A008160809318
:101070007A0080917A00806880937A001092C10093
:1010800084E00E94870085E00E94870087E00E943C
:10109000870060E087E00E94B501E0910902F091CD
:1010A0000A0282E08083E0910502F091060210823C
:1010B000E0910702F091080280E180831092110212
:1010C000E0910D02F0910E0286E08083E0910B0228
:1010D000F0910C02808180618083E0910B02F0919D
:1010E0000C02808188608083E0910B02F0910C02F9
:1010F000808180688083E0910B02F0910C028081F6
:101100008F7D80831092D4011092D3011092A6019A
:101110001092A5010E94910286EA90E09093A201AC
:101120008093A10187EA90E09093A4018093A301AA
:1011300084E48093A4020E94910262EA70E382EA4E
:1011400092E00E945903882331F061E070E080E072
:1011500090E00E94380288E18093B80064E670E075
:1011600080E090E00E9438021E0187E0280E311CCA
:1011700089EF91E00E940601892B09F418C289EFDA
:1011800091E00E94E4008337910509F0DAC166E13D
:1011900074E282EA92E00E945903882309F40CC1A8
:1011A0002FB7F8948091F5019091F601A091F70185
:1011B000B091F8012FBF8093AA029093AB02A09345
:1011C000AC02B093AD022FB7F8948091F5019091E5
:1011D000F601A091F701B091F8012FBF4091AA024A
:1011E0005091AB026091AC027091AD02841B950BE3
:1011F000A60BB70B0597A105B10528F31091A40222
:101200000E9413024B015C018091CD01811166C0E7
:1012100081E08093CD018093CC019FEF9093CB012F
:101220001092CA0195E09093C9018093C801809102
:10123000C801110F182B1093C8018091C70181308C
:1012400009F053C11092C7010E9413024B015C01C7
:101250008091C8018093BB008091CF019091D00113
:10126000A091D101B091D201892B8A2B8B2BA1F0B7
:101270000E9413020091CF011091D0012091D10161
:101280003091D201681979098A099B090617170755
:101290002807390708F443C08091BC0083FDD8CFEC
:1012A000A5ECA093BC000E9413024B015C0180914D
:1012B000CD01813009F41DC18091CA01863008F04A
:1012C0003AC18091CA01A7EAB1E0E5EDF1E090E012
:1012D000981751F12D9121939F5FFACF8091CF0103
:1012E0009091D001A091D101B091D201892B8A2B8C
:1012F0008B2B09F489CF0E9413024090CF015090AC
:10130000D0016090D1017090D201681979098A09E1
:101310009B09461657066806790608F075CF809136
:10132000CE010E94AF0280E01092D4018093D301DD
:10133000863009F002C18E010F5F1F4F8091A2021B
:101340009091A302DC01ED91FC910284F385E02DE4
:101350000995F80181938F012E163F0679F71092B7
:10136000C402898190E0982F88272A81820F911DDD
:101370009093BB028093BA028C8190E0982F8827CB
:101380002D81820F911D9093B9028093B8022FB7DF
:10139000F8948091F5019091F601A091F701B09138
:1013A000F8012FBF8093A6029093A702A093A802F2
:1013B000B093A9021092C4026091B8027091B90270
:1013C00090E080E00E94FD0B28EC30E048EC5AE30E
:1013D0000E94B40C2B013C018090C0029090C1028D
:1013E000A090C202B090C30220E030E0A901C50184
:1013F000B4010E94570B882341F0A5019401C30159
:10140000B2010E94EB0A2B013C016091BA0270917B
:10141000BB0290E080E00E94FD0B2FEA30E04FE23B
:101420005BE30E94B40C20E030E044E352E40E940D
:10143000EA0A4B015C01C090BC02D090BD02E09072
:10144000BE02F090BF0220E030E0A901C701B60162
:101450000E94570B882341F0A7019601C501B401F2
:101460000E94EB0A4B015C0180E10E9401027C01B9
:101470008EE00E9401028C0142E0C301B2010E9491
:10148000C10480E391E00E94700442E0C501B40110
:101490000E94C10480E391E00E947004B701FF0C38
:1014A000880B990B0E94FF0B20E030E040EA5BE3E1
:1014B0000E94B40C42E00E94C10480E391E00E94CB
:1014C0007004B801110F880B990B0E94FF0B20E0EC
:1014D00030E040EA5BE30E94B40C42E00E94C104A9
:1014E00082E391E00E94700443CEB5EEB093BC005D
:1014F000DACE8091CF019091D001A091D101B0912D
:10150000D201892B8A2B8B2B09F4D1CE0E94130296
:101510000091CF011091D0012091D1013091D201E1
:10152000681979098A099B090617170728073907D7
:1015300008F0BDCEF4CE86E0C6CEF2E8F093C40249
:101540003BCF8836910579F461E084E00E94B501D3
:1015500064E670E080E090E00E94380260E084E0A1
:101560000E94B50105CE8936910569F461E085E0F8
:101570000E94B50164E670E080E090E00E943802CD
:1015800060E085E0EDCF8C01015411090A311105AD
:1015900008F0EECD61E0802F0E94B50164E670E0B6
:1015A00080E090E00E94380260E0802FD9CF61E0B7
:1015B00070E080E090E00E94380280E090E0892BAB
:1015C00009F4D6CD0E941201882309F4D1CD0E94DE
:1015D0000000CECD5058BB27AA270E94020B0C94C6
:1015E000750C0E94670C38F00E946E0C20F039F4E4
:1015F0009F3F19F426F40C94640C0EF4E095E7FB7D
:101600000C945E0CE92F0E94860C58F3BA176207FF
:1016100073078407950720F079F4A6F50C94A80CBD
:101620000EF4E0950B2EBA2FA02D0B01B9019001FD
:101630000C01CA01A0011124FF27591B99F0593F41
:1016400050F4503E68F11A16F040A22F232F342F89
:101650004427585FF3CF469537952795A795F040D7
:101660005395C9F77EF41F16BA0B620B730B840BEC
:10167000BAF09150A1F0FF0FBB1F661F771F881FA4
:10168000C2F70EC0BA0F621F731F841F48F48795FC
:1016900077956795B795F7959E3F08F0B0CF9395EE
:1016A000880F08F09927EE0F9795879508950E9467
:1016B0003A0C08F481E008950E94700B0C94750CAC
:1016C0000E946E0C58F00E94670C40F029F45F3FB6
:1016D00029F00C945E0C51110C94A90C0C94640C20
:1016E0000E94860C68F39923B1F3552391F3951B5F
:1016F000550BBB27AA2762177307840738F09F5F33
:101700005F4F220F331F441FAA1FA9F335D00E2E9F
:101710003AF0E0E832D091505040E695001CCAF70C
:101720002BD0FE2F29D0660F771F881FBB1F2617CF
:1017300037074807AB07B0E809F0BB0B802DBF01A6
:10174000FF2793585F4F3AF09E3F510578F00C9475
:101750005E0C0C94A90C5F3FE4F3983ED4F386959D
:1017600077956795B795F7959F5FC9F7880F911D96
:101770009695879597F90895E1E0660F771F881F82
:10178000BB1F621773078407BA0720F0621B730B35
:10179000840BBA0BEE1F88F7E09508950E948E0C1B
:1017A00088F09F5798F0B92F9927B751B0F0E1F022
:1017B000660F771F881F991F1AF0BA95C9F714C0D2
:1017C000B13091F00E94A80CB1E008950C94A80CDF
:1017D000672F782F8827B85F39F0B93FCCF386950B
:1017E00077956795B395D9F73EF490958095709568
:1017F00061957F4F8F4F9F4F0895E89409C097FBE5
:101800003EF490958095709561957F4F8F4F9F4FD7
:101810009923A9F0F92F96E9BB279395F69587951B
:1018200077956795B795F111F8CFFAF4BB0F11F4DE
:1018300060FF1BC06F5F7F4F8F4F9F4F16C0882385
:1018400011F096E911C0772321F09EE8872F762FBB
:1018500005C0662371F096E8862F70E060E02AF0FC
:101860009A95660F771F881FDAF7880F96958795E8
:1018700097F90895990F0008550FAA0BE0E8FEEFBD
:1018800016161706E807F907C0F012161306E40744
:10189000F50798F0621B730B840B950B39F40A263D
:1018A00061F0232B242B252B21F408950A2609F41B
:1018B000A140A6958FEF811D811D089597F99F671F
:1018C00080E870E060E008959FEF80EC08950024C8
:1018D0000A941616170618060906089500240A9495
:1018E00012161306140605060895092E0394000C1B
:1018F00011F4882352F0BB0F40F4BF2B11F460FFAA
:1019000004C06F5F7F4F8F4F9F4F089557FD9058D2
:10191000440F551F59F05F3F71F04795880F97FBB3
:10192000991F61F09F3F79F087950895121613066D
:101930001406551FF2CF4695F1DF08C0161617069C
:101940001806991FF1CF86957105610508940895D1
:10195000E894BB2766277727CB0197F908950E9463
:101960003A0C08F48FEF08950E94C70C0C94750C84
:101970000E94670C38F00E946E0C20F0952311F045
:101980000C945E0C0C94640C11240C94A90C0E9411
:10199000860C70F3959FC1F3950F50E0551F629F21
:1019A000F001729FBB27F00DB11D639FAA27F00DB8
:1019B000B11DAA1F649F6627B00DA11D661F829FDF
:1019C0002227B00DA11D621F739FB00DA11D621FC4
:1019D000839FA00D611D221F749F3327A00D611DE1
:1019E000231F849F600D211D822F762F6A2F1124C3
:1019F0009F5750409AF0F1F088234AF0EE0FFF1FF6
:101A0000BB1F661F771F881F91505040A9F79E3F4C
:101A1000510580F00C945E0C0C94A90C5F3FE4F32C
:101A2000983ED4F3869577956795B795F795E795A2
:101A30009F5FC1F7FE2B880F911D9695879597F9AB
:101A400008950E943A0C880B990B0895A1E21A2E72
:101A5000AA1BBB1BFD010DC0AA1FBB1FEE1FFF1F52
:101A6000A217B307E407F50720F0A21BB30BE40BA2
:101A7000F50B661F771F881F991F1A9469F76095E9
:101A80007095809590959B01AC01BD01CF010895A3
:101A9000EE0FFF1F0590F491E02D0994F894FFCF0D
:101AA000000000004801A800D50095010601E400EF
:101AB000F800000000002703FA025603D002F302E8
:101AC000E002D1026E616E00696E66006F7666009C
:061AD0002C000D0A0000CD
:107E0000112484B714BE81FFF0D085E080938100F7
:107E100082E08093C00088E18093C10086E0809377
:107E2000C20080E18093C4008EE0C9D0259A86E02C
:107E300020E33CEF91E0309385002093840096BBD3
:107E4000B09BFECF1D9AA8958150A9F7CC24DD24C4
:107E500088248394B5E0AB2EA1E19A2EF3E0BF2EE7
:107E6000A2D0813461F49FD0082FAFD0023811F036
:107E7000013811F484E001C083E08DD089C08234E0
:107E800011F484E103C0853419F485E0A6D080C0E4
:107E9000853579F488D0E82EFF2485D0082F10E0AE
:107EA000102F00270E291F29000F111F8ED06801E7
:107EB0006FC0863521F484E090D080E0DECF843638
:107EC00009F040C070D06FD0082F6DD080E0C81688
:107ED00080E7D80618F4F601B7BEE895C0E0D1E017
:107EE00062D089930C17E1F7F0E0CF16F0E7DF06D8
:107EF00018F0F601B7BEE89568D007B600FCFDCFD4
:107F0000A601A0E0B1E02C9130E011968C91119780
:107F100090E0982F8827822B932B1296FA010C0160
:107F200087BEE89511244E5F5F4FF1E0A038BF0790
:107F300051F7F601A7BEE89507B600FCFDCF97BE46
:107F4000E89526C08437B1F42ED02DD0F82E2BD052
:107F50003CD0F601EF2C8F010F5F1F4F84911BD097
:107F6000EA94F801C1F70894C11CD11CFA94CF0C13
:107F7000D11C0EC0853739F428D08EE10CD085E9AC
:107F80000AD08FE07ACF813511F488E018D01DD067
:107F900080E101D065CF982F8091C00085FFFCCF94
:107FA0009093C60008958091C00087FFFCCF809118
:107FB000C00084FD01C0A8958091C6000895E0E648
:107FC000F0E098E1908380830895EDDF803219F02E
:107FD00088E0F5DFFFCF84E1DECF1F93182FE3DFCA
:107FE0001150E9F7F2DF1F91089580E0E8DFEE27F6
:047FF000FF270994CA
:027FFE00040479
:00000001FF
